:100000000C942A000C9434000C9434000C943400AA
:100010000C9434000C9434000C9434000C94340090
:100020000C9434000C9434000C9434000C94340080
:100030000C9434000C9434000C9434000C94340070
:100040000C9434000C9434000C9434000C94340060
:100050000C94340011241FBECFE5D8E0DEBFCDBF25
:100060000E9436000C94F7000C940000CF93DF93AD
:100070001F92CDB7DEB7CE0101960E944A00A59A25
:1000800065E0CE0101960E94B600FACF84B3876086
:1000900084BB08950E944600089585B3887F85BB80
:1000A00085B3962F9370892B6470682B65BB089578
:1000B0002F923F924F925F926F927F928F929F9278
:1000C000AF92BF92CF92DF92EF92FF920F931F9366
:1000D000CF93DF935C01862E942E690100E010E03F
:1000E000212C312C422C532C2AC0C62DD72D682D03
:1000F000C5010E944D002196CF3FD105C1F71016D2
:10010000110654F4C42DD52D692DC5010E944D0052
:100110002196C017D107C1F78FEFE81AF80AEC143F
:10012000FD0421F407C07101602E712E0F3F1105EF
:10013000E4F2E5CF0F5F1F4F0F3F110521F01C14B4
:100140001D048CF3F7CFDF91CF911F910F91FF909A
:10015000EF90DF90CF90BF90AF909F908F907F9067
:100160006F905F904F903F902F900895EC01162F65
:100170002AE030E044E050E067E070E00E94580080
:10018000212F30E046E050E064E070E0CE010E94B4
:100190005800212F30E042E050E066E070E0CE01F0
:1001A0000E945800212F30E043E050E062E070E010
:1001B000CE010E945800212F30E041E050E063E082
:1001C00070E0CE010E945800212F30E045E050E061
:1001D00061E070E0CE010E945800212F30E044E041
:1001E00050E065E070E0CE010E945800C9CFF8945D
:0201F000FFCF3F
:00000001FF
